:02000000662B6D
:08000800F000030EF1000A08EC
:10001000F2000A108A10831237083618B6183E30DC
:1000200081023308B407331C182836083320B4077C
:10003000340CB2003F39B21A403C5520321B103C00
:10004000B2000608F03932048600B60B2B283508BA
:10005000B300B114B6160B1172088A00710E83003A
:10006000F00E700E09008207FF340034FF340034B4
:100070000034FF3400340034FF3400340034FF34E3
:1000800000340034FF3400340034FF3400340034D2
:10009000FF3400340034FF3400340034FF340034C3
:1000A0000034FF3400340034FF348207083408344D
:1000B0000934093409340A340A340A340B340B3451
:1000C0000B340C340C340C340C340D340D340D342E
:1000D0000D340E340E340E340E340E340E340F3410
:1000E0000F340F340F340F340F340F340F348B01AF
:1000F000831650308605831286170130B6008B12A6
:1001000083165730810083128B1308000A300B23AB
:10011000B7000830B50083165830810083128B1663
:100120008B170800B11C92283508031C173CB5003A
:10013000B1100800820755344E34493454347234B7
:10014000613463346B342034763430342E343734B5
:1001500000340339820700346434C8340F3982070D
:1001600000340A3414341E34283432343C344634D7
:1001700050345A34073982072434473450345234C7
:100180004D3443342C3407398207243447345034F7
:100190004734473441342C3482070034003401346E
:1001A000063401340734013403340334003400349A
:1001B000063401340734013401348207003400343A
:1001C00000340134073408340F341034133400344D
:1001D00000340134073408340F3400348207A0346B
:1001E000A034A034A034A034603460342734763492
:1001F00058341C346C3420341C348400B901052973
:1002000084000008A920B900840A0008AE20B907BC
:10021000840A00080F3939070800BA013A08523E2B
:1002200084003A08EE208000BA0A3A080E3A031D0C
:100230000E298A212E218A29B8000930390603198E
:100240003829B908031D45293A08BA203806031D84
:100250003829BA0A2C303806031D08004C308400B7
:1002600030308000840A0408523A031D30297F2967
:100270003A08C3203806031D8A290930B900BA0A92
:100280002C303806031D08007F2938082C3A031942
:100290007F2938082A3A03198A293908CC203A06D6
:1002A000031908003908073A031966290F3A031998
:1002B000662938082E3A031908003908DD203A0764
:1002C0003C3E840038088000BA0A080038082E3AFC
:1002D00003197B293908DD203C3E8400840A00088C
:1002E00084038000840A840A000884038000840A4E
:1002F0003808800008003908CC20BA000800BA018C
:10030000B90A3908093A031989293908103A031D2D
:1003100008008D21BA01B90108003C308400273063
:10032000D9000008413A03199829703A031D9A2907
:100330006030D900BB01840ABA01000DB900153044
:10034000840739081E3960388000EC308407BA0A07
:100350003A08063A031D9D2906300B23BA00C03027
:100360003A1CD406BA1CD3063A1DD206C319D506C8
:100370004418D606CB18D70607300B233038D800E0
:100380000310D80D4530FD201C3EDA004730FD201B
:100390001C3EDB004930FD201C3EDC004C300021BF
:1003A000DE00DD010A30DD0ADE020318D329DD0399
:1003B0005E07AE20DE006C30DD074F3084000008A1
:1003C0000F39203EDE075030FD201C3EDF0047087D
:1003D0000F393C300319DB0745080F39031D0800AE
:1003E0005030DA07D61B08000A30DA07D617561342
:1003F0000800E30D630C922063091F39031D0800F8
:100400000310F9290030052A7E30E1000830E200AF
:10041000E10CF921E301E20B082A080001300B236B
:10042000E000080008300B23E000080086200222CC
:10043000E00B172A0422FF30E400E5000800E10089
:100440000830E200610C01300318E5060310E40CEB
:10045000E50C031C2F2A0830E5068430E406E10C85
:10046000F921E20B222A0800FF30E5066406E000CD
:1004700065081F2260081F22042204227F20080032
:10048000E6000000E60B422A0800831605168511D7
:10049000831285110800E8000A30E7000310851177
:1004A000031C8515A930851E503040220314E80C2A
:1004B000E70B4F2A08000D30642A08000A30642A2E
:1004C00008002030642A08004B2AE900690E6922DE
:1004D00069080F39093C031CF93E393C4B2A681066
:1004E000051E00340930E7003830851E1A304022DE
:1004F0000310051E0314E80CA930851E503040225D
:100500000000E70B782A6808051A842A6814080096
:100510006F22681C882A08008316851086128312B1
:100520000130EC00EB00FF30EE00BB00ED000800F6
:10053000061EED016A080102EA07031C0800031009
:10054000EB0B08002630EB00ED0A0319ED03061E45
:10055000ED01BB0A0319BB03EC0B08000A30EC00E9
:10056000EE0A0319EE0308009822ED080319C22AC7
:1005700005300B236D02031CBF2A8612C32AEB1E13
:100580008612EB1A86163B08053C0318CE2A851006
:100590005908603A27300319D900D82A5908603A17
:1005A0000319D72A6B1A85146B1E8510D82A851457
:1005B0000230061F09300B236E02031CE92A0530A6
:1005C0000B236D020318E52A0A2B0E22EE018A2165
:1005D0000134013E031DFF2AAB1BFD2AAB172B1074
:1005E000AB108A30AA00F9242918FD2A2B1489306F
:1005F000AA00F924291CAB14FD2A86170A2B023005
:10060000061F09300B23053C03180A2B6E08013C1A
:100610000319861300347F3983169B001C141A08B3
:10062000831208007F3983169B008B131C155530ED
:100630009D00AA309D009C141C118B179C181E2B2A
:100640008312080086170515162252308400000810
:100650001F22840A0408593A031D272B00300B235C
:10066000AD002D080B2300380319392B1F22AD0ACA
:10067000312B00081F22840A0408603A031D392B1D
:100680000F300B231F220E300B231F22AC0B562BD7
:1006900003300B23AC0004300B23AD002D080B23DB
:1006A00000380319562B1F22AD0A4E2B3422051198
:1006B00008008514861660238510861260230800C2
:1006C0000000AD0B602BB70B602B080083120730C6
:1006D0009F0045220D2177208C22A5248316051129
:1006E000831205115923592359230130AC00A2016B
:1006F000E32B6F22681C822BAD001B3A0319972B4A
:100700002D081C21B42200380319792B851A2223C5
:10071000851A792B3E24A20A0D300B232202031CDA
:10072000932BA201792BFF30EE00ED01792B88226B
:10073000AD001B3A0319972B2D08443A0319CD2B12
:100740002D08553A0319D92B2D08563A0319E32BD6
:100750002D08313A0319ED2B2D08323A0319F02BED
:100760002D08333A0319FA2B2D08523A0319022C9B
:100770002D08723A0319222C2D08773A03190B2CF5
:100780002D08753A03199B2C2D08423A03190E2D9A
:100790002D08493A0319A524792BAD018822831627
:1007A0009A0083122D081223AD0AAD1FCE2B8C2286
:1007B000792B80306422AD012D080B236422AD0A11
:1007C000AD1FDC2B792BAD012D089A2000380319C1
:1007D000EC2B6422AD0AE42B792B05158620F42B33
:1007E00005158620031092206F22681CF42B7F20B1
:1007F0000511792B05158620031092206F22681CA5
:10080000FC2BF72BAD012D08840000086422AD0AF3
:10081000031D032C792B83162130A00020088400AF
:10082000831288228316841780008413A00A201F55
:100830001D2CA01E1D2C201A202C0D3A031D0E2C41
:100840008312792B83162130A0002008840084179E
:1008500000088413831264228316A00A201F342CFC
:10086000A01E342C201A3A2C8417000884130D3A49
:10087000031D252C83125B225E22792B861705151A
:10088000162282301F22A0301F228A301F22AE3053
:100890001F22B0301F2260301F2260301F22003024
:1008A0000B23AD002D080B23003803195A2C1F22EF
:1008B000AD0A522C0B300B23AD002D080B23003852
:1008C0000319652C1F22AD0A5D2C83162130A00070
:1008D000200884008417000884130D3A03197D2C26
:1008E00084170008841383121F228316A00A201F76
:1008F000682CA01E682C201E682C83120C300B2341
:10090000AD0058301F2250301F224930AB186930DB
:100910001F2243302B1863301F2220301F222D0846
:100920000B2300380319972C1F22AD0A8F2C342279
:100930000511AB13080080306422AD012D080B2394
:100940006422AD0AAD1F9E2C792B213084008417C0
:1009500030308000840A8000840A8000840A2F30AE
:100960008000840A30308000840A8000840A80007D
:10097000840A67308000840A30308000840A800056
:10098000840A8000840A74308000840A3030800039
:10099000840A8000840A8000840A2F308000840A40
:1009A0004E308000840A6F308000840A5730800007
:1009B000840A58308000840A64308000840A6130E0
:1009C0008000840A74308000840A61308000840AC8
:1009D00020308000840A0D3080008413080000005D
:1009E0000000000000000000000000000000000007
:1009F000003412309F00EF242A0883169F008312D0
:100A0000EF241F1B29141F1F291007309F00EF24FC
:100A100083160F309F008312EF240034AB01AD0129
:100A200086168A30AA00F92429188616291C8612EF
:100A3000AD03031D112DAB03031D112D5B225E229F
:040A40008612792B76
:02400E00020DA1
:1042000010002800010001004500020000003000FD
:1042100028003C0040002100360001002F00620011
:104220009C009E00860082009800980060009C0020
:104230009E00A0008200A800900061000300F00032
:104240000000210035003000300030002E0030002A
:1042500030004E002F0030003100340033003000B9
:104260002E003000300045005F000000570058006D
:1042700054007200610063006B00200076002E0085
:10428000200030002E003700000055006E0069004D
:1042900054007200610063006B00200076002E0065
:0E42A000200030002E0037000000000000005B
:00000001FF
